:10000000000C0600FF0C05006C00EC000C02260042
:1000100068006800040C88000306480A7109A802F9
:100020000B02C00FC00E43070A0A0B0230008C05FA
:100030008B064C048B074C05AB06CC04AB07CC05F8
:100040007109800CAB010B02C00E4307480A710016
:100050001007D1041006D1053007F1043006F10570
:100060000B0231017109800CAB010B02C00E43077A
:10007000480A72005007D2045006D2057007F204F5
:100080007006F2050B0232017202B2026800090A20
:10009000060C88000306090A7109A8020B02800FEA
:1000A000F80E4307480A0B02300071090B023100B9
:1000B00071090B02320071090B02310071090B0248
:1000C000320010074C0410064C0530078C04300633
:1000D0008C055007CC045006CC050C0226006800A5
:1000E000480A2506740A710A080C2A0082098E093A
:1000F00025070304250603052B03EA02770A6B0292
:10010000820900087D0C29000000000000000000AA
:10011000000000000000E902840A00082D0C2900FC
:1001200011024306A80AF106BB0A00000000000005
:1001300000000000F1000C06A10AAC06A60A0C059E
:10014000B60AAC060C04AC07AC05B80AAC04B70A96
:10015000000000000000000000000000000000009F
:10016000000000000000000000000000000000008F
:100170000C022600D30A7102B10200000000F10057
:10018000AC06C60A0C06CB0AAC05CD0A0C06AC04BC
:100190000C070C05CF0A0C04CE0A000000000C026C
:1001A00026007102B10212024306EB0AF206FE0AB1
:1001B00000000000000000000000F200EC06E40A6D
:1001C0002C06E90AEC05F90A2C06EC042C072C0590
:1001D000FB0A2C04FA0A00000000000000000000E6
:1001E000000000000000000000000000000000000F
:1001F0000000000000000C022600160B7202B20282
:1002000000000000F2002C06090BEC060E0B2C057A
:10021000100BEC062C04EC07EC05120BEC04110B94
:10022000000000000C0226007202B202E902900AED
:100230000008FF0FFF0FFF0FFF0FFF0FFF0FFF0F54
:00000001FF
